:1000000009C00EC00DC00CC00BC00AC009C008C09A
:1000100007C006C011241FBECFE9CDBF02D02FC03C
:10002000EFCF81E02DE387BB28BBB199FCCF98B31C
:10003000982798BBEFE7F2E03197F1F700C0000096
:1000400098B3982798BBEFEBF4E13197F1F700C034
:10005000000098B3982798BBEFE7F2E03197F1F7EB
:1000600000C0000098B3982798BBFFEF3FE341E042
:10007000F15030404040E1F700C00000D4CFF89488
:02008000FFCFB0
:00000001FF
